S01900006F70656E626C745F73746D3332673037312E7372656300
S31508000000600900204D1B0008BB07000843080008CC
S3150800001000000000000000000000000000000000D2
S315080000200000000000000000000000009B08000817
S3150800003000000000000000004709000899080008B1
S31508000040571300083F1800082B1B0008371B000829
S31508000050791B00087B1B00087D1B00087F1B000816
S31508000060811B0008831B0008851B0008871B0008E6
S31508000070891B00088B1B00088D1B00088F1B0008B6
S31508000080911B0008931B0008951B0008971B000886
S31508000090991B00089B1B00089D1B00089F1B000856
S315080000A0A11B0008A31B0008A51B0008A71B000826
S315080000B0A91B0008AB1B0008AD1B00080020C043A5
S315080000C06D4908606D490860704770B504000D00F9
S315080000D016006B48001B691E88420AD3200000F0F0
S315080000E09EF9FF2805D06019401E00F098F9FF28F0
S315080000F001D1002070BD3200600A40026149884281
S3150800010005D12B0021005D4800F0BEF870BD2B001C
S315080001102100594800F0B8F870BDF8B504000F0082
S315080001200126FF2005005649091B7A1E914200D276
S315080001300026310001290ED1200000F070F90500D3
S31508000140E019401E00F06BF92900FF2902D00100D2
S31508000150FF2900D100263100012904D10100280019
S3150800016000F00DF906003000F2BD012043490A6887
S315080001700023DB439A4200D1704780B548688A68F5
S315080001808018CA6880180A6980184A6980188A69B6
S315080001908018C9694018C143491C00916A46042160
S315080001A0B948FFF792FF02BD012036490A684B6835
S315080001B0D2188B68D218CB68D2180B69D2184B693B
S315080001C0D21889695118B04A1268891800D00020D7
S315080001D0704738B501240025ED4328480168A9422F
S315080001E004D000F09BF8002800D100242000012844
S315080001F008D121480168A94204D000F08FF80028E8
S3150800020000D10024200032BD1E48704710B50124D5
S31508000210CA0500D000242200012A08D102688A42B1
S3150800022005D0016080229200001D00F071F92000BF
S3150800023010BDF8B506000F00002425000F488642B9
S3150800024002D10D4D2E000BE00E498F4202D1060059
S31508000250050005E0300000F061F8012800D13500FE
S31508000260002D06D039003000FFF7D0FF002800D156
S3150800027025002800F2BD000090000020940200200E
S31508000280FFFF010800200008F7B504000E001F0054
S315080002900125700A4002019020680021C94388425E
S315080002A006D101992000FFF7B1FF002800D10025EB
S315080002B02800012809D120680199884205D0200024
S315080002C0FFF7B7FF040000D100252800012823D135
S315080002D002982168711A61180E1D69460D7005008D
S315080002E000F02AF980208000211D711A814207D367
S315080002F0019909182000FFF79CFF040007D0261D66
S3150800030028783070761C6D1C7F1EE9D102E000202B
S3150800031069460870684605782800FEBDFEB50700E0
S315080003200126386800F07BF8FF2800D10026300047
S31508000330012822D100F03AF9002400E0641C402C80
S3150800034019D2E00039680D183818001D03C86A4626
S3150800035003C200F0F1F868460CC82900012000F035
S31508000360F7F8002806D10CCD684603C88B4201D1A0
S315080003708242E3D0002600F027F93000FEBDF0B532
S3150800038085B00F0001252C00002101913A000300D9
S315080003909A4200D20C002200012A06D10200042A41
S315080003A002D33A00132A00D30C002100012933D1C5
S315080003B000F04FF80600380000F04BF801000091F5
S315080003C0380000F063F800990818401E801B401C8E
S315080003D0C00A80B2009002200290F8200006301869
S315080003E0C00A0390049500F0E1F800273D00009E3E
S315080003F003E00398401C03906D1C280080B2B042AD
S3150800040008DA00F099F801A902A800F03BF90028DB
S31508000410EFD03C0000F0D8F8200005B0F0BD38B5A4
S315080004200400002501E06D1CEDB20F2D0FD200F07F
S3150800043083F82348690049198900401801688C42E5
S31508000440F1D3426889188C42EDD2007A32BDFF207A
S3150800045032BD38B50400002500E06D1C2800C0B286
S315080004600F280ED200F068F815482900C9B24A00CC
S31508000470511889004018017A22009142EDD100688E
S3150800048032BD0020C04332BDBC20000838B5040088
S31508000490002500E06D1C2800C0B20F280ED200F01F
S315080004A04BF807482900C9B24A0051188900401874
S315080004B0017A22009142EDD1406832BD002032BD5A
S315080004C09818000880B500F035F901BD10B500F0A0
S315080004D041F9002816D000F057F9002812D000F08C
S315080004E086F900F0BCF900F0EBF900F037F9064997
S315080004F001400648016000F031F9001D046800F06B
S315080005001BF9A04710BD000080FFFF1F08ED00E0A3
S3150800051070B515000C00060005E020783070641CE4
S31508000520761C00F009F82800451E0004F5D170BDB8
S3150800053080B500F039F901BD80B500F03AF901BD82
S3150800054008B4024B9C4608BC6047C04655000020CC
S31508000550F1B50F0014001D0043480078012801D1A9
S315080005600220F2BD01204049087000260846466070
S31508000570FA20800000F034F8010014D13800220077
S315080005802B000099012902D100F060F802E0110061
S31508000590FFF7D6FFFA20800000F022F833490A68F0
S315080005A0009B9A430A6030490E70F2BD002032491A
S315080005B0CA68002A07D5314A0A60314A0A60C968FA
S315080005C0002900D501207047012028490A688023A0
S315080005D01B0613430B600968002900D500207047E5
S315080005E070B5040000F054F90619214D2868C003B7
S315080005F005D500F04DF9B042F8D3032070BD286840
S315080006001C490140A8688022D20510400843810F82
S31508000610890704D0A968820F92070A43AA60810055
S31508000620890800D02960002803D00F4948600120B6
S3150800063070BD00F02DF904192868400304D500F0B0
S3150800064027F9A042F8D3D8E7002070BD30B407498F
S315080006500C68012525430D600260BFF36F8F001DEE
S31508000660036030BC704700003005002014200240AB
S3150800067010200240FAC30000082002402301674503
S31508000680AB89EFCDF8B505000E002548007801289E
S3150800069001D10220F2BD0120214908700024084634
S315080006A04460FA208000FFF79BFF010025D12968E6
S315080006B0042906D100F024F8FA208000FFF790FFFD
S315080006C01BE00021C9433160696837000E0000E06D
S315080006D0761C6968AA6889188E4209D2300000F02B
S315080006E015F8FA208000FFF77BFF0100F0D03E6086
S315080006F00C490A6802239A430A6009490C70F2BD3C
S3150800070008480168084A0A430260704705490B68A9
S31508000710064A1A40C0001043054A02430A60704759
S3150800072030050020142002400400010007FEFFFFE8
S315080007300200010072B6704762B6704780B5FFF7CF
S31508000740BDFC01BD80B5FFF7C0FC02BD80B5FFF753
S31508000750E4FC02BD80B5FFF727FD02BD80B5FFF7B3
S3150800076053FD02BD80B5FFF700FD002801D100202A
S3150800077002BDFFF72EFD02BD00690840884201D17F
S31508000780012070470020704780B5802189010548FF
S31508000790FFF7F2FF002801D1002002BD00F0CCF8D7
S315080007A0012002BD0008005080B5642000F0A2F8C0
S315080007B001BD80B500F0A1F801BDFEE780B500F0E7
S315080007C0C3F800F0ABFA00201849087001BD1CB543
S315080007D0164C6946201D00F0D6FA012806D10020DD
S315080007E0207068460178201D00F0C9F813BD7047CF
S315080007F080B50E4A1278002A02D1C9B200F0A6FACC
S3150800080000F0B9F801BD09480078401E022801D851
S31508000810002070474020704704480078401E022890
S3150800082001D80020704740207047000000000020D3
S3150800083010B5002400F098F8002800D00124200004
S3150800084010BDFEE780B500F00AF80E480E49416073
S3150800085000218160052202600C48016001BD00206C
S3150800086008490860704707480068C00303D5074869
S315080008700168491C0160704780B5FFF7F4FF03481B
S31508000880006802BD10E000E0FFF900005C050020EA
S3150800089080B5FFF7F1FF02BD7047FEE710B50024EB
S315080008A010480168820D0A430260204600F0D6FA15
S315080008B0002801D0012401E000F0D1FB200010BD82
S315080008C080B509480021C943816000228260C16061
S315080008D0C260416042600160026000F0FBFB0020DC
S315080008E002BD0000002002402410024081617047CA
S315080008F0816270470F494880704710B5FFF7BCFF03
S315080009000C4C6168884214D3A020C00521780029C0
S3150800091005D1012121702021FFF7E8FF04E000211D
S3150800092021702021FFF7E4FFFFF7A6FF6188401832
S31508000930606010BD5405002080B52021A020C005A8
S31508000940FFF7D6FF01BDFEE710B40020BB49020041
S315080009500A800A0044325060030043240B55138072
S3150800096002008A7010BC7047B4480078401E804167
S31508000970C043C00F70470020B1490870704710B5D2
S31508000980AE4C0178FF2914D100F086F84320205C8C
S31508000990012802D1102000F077F84420215E0800D3
S315080009A0012805DB01204322A054E01C00F050F882
S315080009B010BD21780129FBD10178C92932D0CC296B
S315080009C03FD0CF293AD0D0292FD0D12933D0D22918
S315080009D02ED0F32917D0F4290FD0F5290AD0F629F5
S315080009E00ED0FA2912D0FC2913D0FD2914D0FE29DD
S315080009F015D029E000F0A6F8C8E700F0C1F8C5E769
S31508000A0000F097F8C2E700F0DAF8BFE700F080F8E0
S31508000A10BCE700F078F8B9E700F068F8B6E700F048
S31508000A2059F8B3E700F0ECF8B0E700F00BF9ADE7DA
S31508000A3000F0D7F8AAE700F032F9A7E700F042F984
S31508000A40A4E700F04BF9A1E7202000F01DF89DE788
S31508000A5080B589B2FFF7CCFE01BDF8B517000026B0
S31508000A6004000D0004E020783618641CFFF764FDC6
S31508000A702800451E0028F6D1F6B23E600120F2BDD8
S31508000A8000206E49487070476C49FE22CA7008718A
S31508000A90022044228852704738B5FFF7F1FF674CA9
S31508000AA001252570FF20E07010202071002060715C
S31508000AB0FFF7A9FEA071FFF7AFFEE071FFF7ACFEE6
S31508000AC0000A20726572A572082044216052FFF759
S31508000AD035FE31BD10B5594C00202070FFF7D0FF08
S31508000AE0FF20E07001204421605210BD5348FF21C9
S31508000AF0C1700021017142784271C18001720621DC
S31508000B0044228152704780B50020FFF7BDFF01BD22
S31508000B104A48FF21C1700100443100BF72A24A60F1
S31508000B200022828082710722C01C42600820088049
S31508000B3070474249FF22CA70443140684860012024
S31508000B400880704770B50500FFF75DFE6A78401E9D
S31508000B501100884203DA2220FFF796FF70BD374C52
S31508000B60260044367168201DFFF7D2FCFF20E0708E
S31508000B7070686978401870606878401C308070BD6D
S31508000B8070B50400FFF73FFE401E6178884203DA1D
S31508000B902220FFF779FF70BD6168284D2E00443684
S31508000BA071606278281DFFF7B3FCFF20E870706853
S31508000BB06178401870606078401C308070BD38B528
S31508000BC01E4CFF21E17025004435E21D4168686826
S31508000BD0FFF743FF207100206071A071082028806C
S31508000BE031BD38B5154CFF20E0700025A580FFF70C
S31508000BF00AFEA071E571258107204421605231BDA6
S31508000C0070B50600FFF7FFFD0C4C25004435721C35
S31508000C10411E6868FFF796FD002803D13120FFF7CB
S31508000C2033FF70BDFF20E070FFF7EDFD6968401ED9
S31508000C30081868600120288070BD0000E4040020C0
S31508000C402705002038B50400FFF7DDFD801E617812
S31508000C50884203DA2220FFF717FF31BD1E48FF211D
S31508000C60C17005004435012028806178002907D124
S31508000C70FFF778FD002811D13120FFF705FF31BDB8
S31508000C80A21C6868FFF75EFD002803D13120FFF734
S31508000C90FBFE31BD686861784018686031BD38B5BB
S31508000CA00D4C2500443541686868FFF74FFD00285C
S31508000CB003D13120FFF7E8FE31BDFF20E0700120A7
S31508000CC0288031BD80B5FFF701FC0348FF21C170BC
S31508000CD001214422815201BDE404002080B531205F
S31508000CE0FFF7D2FE01BD00004F70656E424C5400FE
S31508000CF0016801220A4302607047C0694109080079
S31508000D00C007C00F7047C069C1090800C007C00FF7
S31508000D107047406AC0B270478162704710B588B0A4
S31508000D20E1200002019000200290039004900C211B
S31508000D300591069007900090454C6946200000F002
S31508000D4047FA2000FFF7D4FF08B010BD70B50500BC
S31508000D500C002000412803DB74213E4800F0A0FA6D
S31508000D60200000F05EF8002607E0FFF7E5FB3000FC
S31508000D7080B2285C00F055F8761C3000210080B25D
S31508000D808842F2D370BDF8B507000D00324C607882
S31508000D90002811D1201D00F034F801282FD1207920
S31508000DA000282CD041282ADAFFF766FDA064002027
S31508000DB020700120607022E02678601D31004018FE
S31508000DC000F01FF8012812D1761C3200227010009C
S31508000DD02179C0B2884212D13800D2B2611DFFF71C
S31508000DE097FB00206070207828700120F2BDFFF77D
S31508000DF043FDA16C6431814201D20020607000205D
S31508000E00F2BD70B504000025114E3000FFF775FFDE
S31508000E10002804D03000FFF77CFF20700125280049
S31508000E2070BD38B501000A4C2000FFF775FFFFF7C3
S31508000E3023FD05000A352000FFF765FF002805D1C8
S31508000E40FFF77AFBFFF718FD8542F4D231BD0000A3
S31508000E5000440040A01900089804002070B5060058
S31508000E600024114DA96800291AD0FA20800000F044
S31508000E701BFA01000D48006800F016FA00F0A7FA00
S31508000E8000280BD1042E07D2224631000020C04389
S31508000E9000F099FA6E6004E0012402E0012400E003
S31508000EA00124200070BD00BF44000020500000202F
S31508000EB099480168820D0A4302607047964800689F
S31508000EC0810A0800C007C00F704794490A680723BB
S31508000ED09A431043086070479048016838200840D4
S31508000EE070478E490A688E4B13401843086070474E
S31508000EF08A490A688B4B134018430860704786482E
S31508000F000168802252040A430260704782480068DA
S31508000F10410E0800C007C00F704770B4824C2568A0
S31508000F20824E2E4030430143100208430343236098
S31508000F3070BC70477C480168802252050A430260EB
S31508000F40704781B07A490A6802430A60096808400E
S31508000F500090009801B0704775490A6882430A6094
S31508000F60704781B073490A6802430A6009680840F5
S31508000F700090009801B070476E490A6882430A607B
S31508000F80704781B06C490A6802430A6009680840DC
S31508000F900090009801B0704767490A6882430A6062
S31508000FA0704781B065490A6802430A6009680840C3
S31508000FB00090009801B0704760490A6882430A6049
S31508000FC070475F490A6807239A43104308607047C9
S31508000FD05B4800684007400F70478162704780B5DC
S31508000FE000F005F800F0FEF900F00AFAFCE780B513
S31508000FF0FFF754FC00F001F801BD80B50220FFF7A9
S31508001000E0FFFFF7E5FF022803D066214D4800F010
S3150800101047F9FFF74DFFFFF751FF0128FBD1C02322
S31508001020DB05402230210220FFF777FFFFF767FF35
S31508001030FFF780FFFFF76AFF0128FBD10020FFF7C3
S3150800104050FF0020FFF754FF0220FFF73EFFFFF78F
S3150800105043FF1028FBD13C4800F0DCF901BD70B510
S3150800106086B00120FFF78DFF80204000FFF769FF5B
S315080010700120FFF796FF0420FFF793FF80208002E8
S31508001080FFF76FFF202000900124019400250295A8
S3150800109003950495A026F6056946300000F049FA3E
S315080010A020213000FFF799FF600300900195049511
S315080010B06946264800F03DFA0C200090022001906F
S315080010C002950395049505946946300000F031FAB7
S315080010D006B070BD10B500F0C9FAA024E4052021B9
S315080010E02000FFF77AFF194800F0EBF9200000F01E
S315080010F0E8F980208002FFF73FFF0420FFF75CFF36
S315080011000120FFF759FF80204000FFF725FF012047
S31508001110FFF742FF10BD0000001002400810024011
S31508001120FFF0FFFFFF8FFFFF0C1002408C80FF1FB0
S31508001130381002403C100240401002403410024071
S31508001140002002404C1900080090D0030008005007
S3150800115001680800C007C00F7047C26A0F239A4388
S3150800116089B20A43C262704742683F4B134019432B
S315080011704160704782683D4B134019438160704750
S315080011800000000070B504001D00049E080000BFA2
S315080011903DA192B25200895A00F086F87108802261
S315080011A0120295420DD140004018310000F07CF83B
S315080011B080B22F49014040084007400F0143E160D3
S315080011C070BD4018310000F06FF880B2E06070BD65
S315080011D0F8B584B005000E0001270024FFF7B8FF14
S315080011E000283ED1286827490140B068084331697C
S315080011F0014370690843F16901432960F1682800D1
S31508001200FFF7B2FFB1692800FFF7B4FF1948854216
S3150800121004D1032000F056FA040011E0164885426E
S3150800122004D10C2000F04EFA040009E01348854268
S3150800123002D01348854203D101A800F037FA039C6F
S31508001240002C0AD07068002807D000270090F369A0
S31508001250326821002800FFF795FF31682800FFF75C
S315080012607CFF380005B0F0BDFFCFFFFFFFFCFFFF96
S31508001270F0FF0000003801400044004000480040EC
S31508001280004C0040F369FFEF01000200040006006D
S3150800129008000A000C001000200040008000000131
S315080012A080B5FFF749F9FCE70022030A8B420BD207
S315080012B003098B4219D243088B422ED2411A00D217
S315080012C00146524110467047FF2209023FD01206D6
S315080012D08B4205D3121209028B4201D3121209025C
S315080012E003098B4219D300E0090AC3098B4201D3CB
S315080012F0CB01C01A524183098B4201D38B01C01A14
S31508001300524143098B4201D34B01C01A524103098A
S315080013108B4201D30B01C01A5241C3088B4201D339
S31508001320CB00C01A524183088B4201D38B00C01AE6
S31508001330524143088B4201D34B00C01A524188429E
S3150800134000D3401A5241CFD201461046704708B51D
S3150800135000F074FA08BDFEE710B4C2001823134063
S31508001360FF249C40E2438901C9B2994003000BD58A
S31508001370194B0007000F0838800880001818036802
S315080013801A401143016007E014489B089B00C018E7
S3150800139003681A401143016010BC704710B5401E1F
S315080013A080214904884201D3012010BD0C4C60609D
S315080013B003210020C043FFF7CFFF0020A0600720CD
S315080013C02060002010BD80B5FFF7C6FF01BD80B5BF
S315080013D0FFF7E4FF02BD00001CED00E000E400E0BA
S315080013E010E000E080B5FFF76DF8FFF7A1F8FFF70A
S315080013F029FAFFF7A3F9FFF7E1F900F021FA01BD91
S3150800140080B5FFF799F8FFF72EFAFFF7E0F900F035
S3150800141020FA01BD0149086070470000500000200D
S3150800142010B40B004B4301685C00E418A143534316
S315080014300B43036010BC704743688B435143194301
S315080014404160704710B40B004B4381685C00E41898
S31508001450A14353430B43836010BC704710B40B0081
S315080014604B43C1685C00E418A14353430B43C36074
S3150800147010BC704710B40B004B434B434B43016AF7
S315080014801C01E41AA14353430B43036210BC704783
S3150800149010B4090A0B004B434B434B43416A1C01EA
S315080014A0E41AA14353430B43436210BC70473F49B8
S315080014B00A681043086070473C490A6882430A6014
S315080014C0704710B50024A021C905884206D101201D
S315080014D0FFF7EDFF0120FFF7EFFF28E034498842C8
S315080014E006D10220FFF7E3FF0220FFF7E5FF1EE023
S315080014F03049884206D10420FFF7D9FF0420FFF7B8
S31508001500DBFF14E02C49884206D10820FFF7CFFFFD
S315080015100820FFF7D1FF0AE02849884206D1202093
S31508001520FFF7C5FF2020FFF7C7FF00E001242000D2
S3150800153010BDF8B5002607000D0027E02100380089
S31508001540FFF7A6FF21E00124B4400C401DD06A68CD
S3150800155021003800FFF764FF6868012801D00228D7
S3150800156004D1AA6821003800FFF76CFF2A69210018
S315080015703800FFF773FF6868022806D16A69FF2CEE
S31508001580DCD821003800FFF775FF761C29680800AB
S31508001590F040D8D138006A68012A01D0022A02D15F
S315080015A0EA68FFF749FF0020F2BD00002410024058
S315080015B00004005000080050000C005000140050B1
S315080015C066480068410C0800C007C00F70476348AA
S315080015D00168820D0A430260704760480068810A04
S315080015E00800C007C00F70475D490A685D4B134085
S315080015F000021843086070475B4800684108080005
S31508001600C007C00F7047594801683820084070471E
S3150800161056480168F02000010840704753480168A1
S31508001620E020C0010840704751490968014000049C
S315080016300843704749480068410E0800C007C00FB4
S3150800164070474C480068000A4006400E70474948F3
S315080016500068400F40077047464800688007800FBB
S3150800166070474448016870200840704770B5FFF716
S31508001670AEFFFFF7B2FF0128FBD14020FFF7B4FF0A
S31508001680364C0025A560A60D2660FFF799FF0028B1
S31508001690FBD12660FFF7CEFF0028FBD1A00CE06047
S315080016A0A5610020C0432062284670BD10B504001D
S315080016B000F068F8206000F07DF8606000F089F8B6
S315080016C0A06010BD10B5002403281FD10320FFF722
S315080016D0ABFF2949401A26D0401E02D0401E06D02C
S315080016E00CE0FFF77AFF012835D1244C33E0FFF7E9
S315080016F083FF01282FD1802424022CE000F042F831
S3150800170000F058F800F065F8040024E00C2822D10F
S315080017100C20FFF789FF1A49401A04D0001F06D08B
S31508001720001F0AD010E000F02DF8040013E0FFF7C0
S3150800173054FF01280FD1114C0DE0FFF75DFF01287A
S3150800174009D18024240206E000F01CF800F032F8E3
S3150800175000F03FF80400200010BD00000010024011
S3150800176004100240FF80FFFF5C1002400810024090
S31508001770541002400C100240010003000024F4003B
S3150800178004000C0080B5FFF73EFF082802D0102899
S3150800179002D004E0254802BD00F029F802BD012167
S315080017A023480068C00A4007400F81401E48FFF7DB
S315080017B07BFD02BD10B50400FFF72AFF1D49000A8C
S315080017C00007000F8000085CC006C00EC440200059
S315080017D010BD10B50400FFF721FF1749000B800064
S315080017E0085CC006C00EC440200010BD000010B53D
S315080017F0FFF732FF032801D10C4C00E00A4CFFF733
S3150800180020FF4443FFF72DFF010020000909491C6A
S31508001810FFF74AFD0400FFF71AFF410F491C200095
S31508001820FFF742FD10BD00000024F40000127A0004
S3150800183000100240E0190008E01A00087047FEE7A9
S3150800184080B501201349087000F01BF800F001F874
S3150800185001BD10B5FEF7ECFF012811D00D4C20781C
S3150800186001280DD1FFF708F8A16862688918FA22DD
S3150800187052008918884203D300202070FEF726FEFE
S3150800188010BD10B5034C2078012802D1FEF7F4FFED
S31508001890606010BD48050020002000080008000010
S315080018A004000000002800080008000005000000E9
S315080018B00030000800080000060000000038000894
S315080018C000080000070000000040000800080000AB
S315080018D00800000000480008000800000900000091
S315080018E000500008000800000A0000000058000820
S315080018F0000800000B000000006000080008000057
S315080019000C00000000680008000800000D00000038
S3150800191000700008000800000E00000000780008AB
S31508001920000800000F00000000800008008000008A
S3150800193010000000000001080080000011000000EF
S31508001940008001080080000012000000433A5C573E
S315080019506F726B5C736F6674776172655C4F7065E6
S315080019606E424C545C5461726765745C44656D6F75
S315080019705C41524D434D305F53544D333247305FCF
S315080019804E75636C656F5F4730373152425F494128
S31508001990525C426F6F745C6D61696E2E6300000065
S315080019A0433A5C576F726B5C736F667477617265E6
S315080019B05C4F70656E424C545C5461726765745C2A
S315080019C0536F757263655C41524D434D305F535496
S315080019D04D333247305C72733233322E6300000067
S315080019E000000000000000000000000000000000E9
S315080019F000000000000000000000000000000000D9
S31508001A0001000000020000000300000004000000BE
S31508001A10060000000700000008000000090000009A
S31508001A2070B40123002413E00168001D194202D096
S31508001A304D466D1E49190C60091D121F042AFAD25B
S31508001A400D00960701D50C80AD1C1A4000D02C70ED
S31508001A500268001D002AE7D170BC704730B50168DE
S31508001A604118446862088A188368E40704D54C4616
S31508001A701B1901E0641C06D191420BD00C7864B2A4
S31508001A80491C0D78491C1D705B1C002CF2D4641E81
S31508001A90F7D5F1E70C3030BD10B507497944183150
S31508001AA0064C7C44163404E0081D0A6889188847E1
S31508001AB00100A142F8D110BD080000002400000072
S31508001AC061FFFFFFD0040000900000200000000026
S31508001AD08DFFFFFFDA0000009800000000000020DC
S31508001AE000000000000000000000000000000000E8
S31508001AF001000000020000000300000004000000CE
S31508001B0000F00DF8002801D0FFF7C6FF00BF00BFA0
S31508001B10002000BF00BFFFF762FA00F002F80120BC
S31508001B20704780B500F002F801BDFEE70746384663
S31508001B3000F002F8FBE7FEE780B500BF00BF024AE7
S31508001B4011001820ABBEFBE72600020001488047BB
S31508001B50014800475D1B00086D1B00088020000532
S31508001B60014908607047000008ED00E000BF00BFAB
S31508001B7000BF00BFFFF7C4FFFEE7FEE7FEE7FEE78C
S31508001B80FEE7FEE7FEE7FEE7FEE7FEE7FEE7FEE71F
S31508001B90FEE7FEE7FEE7FEE7FEE7FEE7FEE7FEE70F
S31508001BA0FEE7FEE7FEE7FEE7FEE7FEE7FEE70004E0
S31508001BB0B9000004FD000001FC003E24F40030B426
S31508001BC000230C4A54688025ED0225435560EFF33F
S31508001BD0108472B604E00D680560091D001D5B1CC3
S31508001BE01D00EDB2402DF6D31068C003FCD484F373
S30F08001BF0108830BC70471020024030
S70508001B6D6A
